:100000000C94A3070C94DD070C94DD070C94DD071A
:100010000C94DD070C94DD070C94DD070C94DD07D0
:100020000C94DD070C94DD070C948F2A0C94652B3F
:100030000C94C8240C94DD070C94DD070C94DD07A8
:100040000C94DD070C94DD070C94DD070C94DD07A0
:100050000C94DD070C9450250C94DD070C94DD07FF
:100060000C94DD070C94DD070C94DD070C94DD0780
:100070000C94DD070C94DD070C94DD070C94DD0770
:100080000C94DD070C94DD070C94DD070C94DD0760
:100090000C94DD070C94DD07C30CC30CEF0CEF0CC4
:1000A000570D750D8D0E8D0E800D190E2A0E2A0E10
:1000B000D62BFD2BF52CFD2BF52C492C6C2CF52C7F
:1000C000C32CD22C68747470733A2F2F716D6B2E01
:1000D000666D2F01012800514D4B20697320746813
:1000E000652062657374207468696E672065766543
:1000F00072210029003A003B003C003D003E003FD9
:1001000000000000000000400041004200430044A5
:10011000004500460053004A00010035001E001F44
:100120000020002100220023005400550056002426
:10013000002500260027002D002E002A0000004D7B
:10014000004B002B0014001A000800150017005F78
:10015000006000610057001C0018000C0012001322
:10016000002F00300031004C004E00390004001612
:1001700000070009000A005C005D005E0000000B43
:10018000000D000E000F00330034000000280000B6
:10019000000000E1001D001B0006001900050059C9
:1001A000005A005B0058001100100036003700387C
:1001B000000000E500000052000000E000E300E263
:1001C000002A002C00000062000000630000002AEA
:1001D000000000E600E70065000000E40050005168
:1001E000004F0029003A003B003C003D003E003F2C
:1001F00000000000000000400041004200430044B5
:10020000004500460053004A00010035001E001F53
:100210000020002100220023005400550056002435
:10022000002500260027002D002E002A0001004D89
:10023000004B002B0014001A000800150017005F87
:10024000006000610057001C0018000C0012001331
:10025000002F00300031004C004E00390004001621
:1002600000070009000A005C005D005E0000000B52
:10027000000D000E000F00330034000000280000C5
:10028000000000E1001D001B0006001900050059D8
:10029000005A005B0058001100100036003700388B
:1002A000000000E500000052000000E000E300E272
:1002B000002A002C00000062000000630000002AF9
:1002C000000000E600E70065000000E40050005177
:1002D000004F0029003A003B003C003D003E003F3B
:1002E00000000000000000400041004200430044C4
:1002F000004500460053004A00010035001E001F63
:100300000020002100220023005400550056002444
:10031000002500260027002D002E002A0000004D99
:10032000004B002B0014001A000800150017005F96
:10033000006000610057001C0018000C0012001340
:10034000002F00300031004C004E00390004001630
:1003500000070009000A005C005D005E0000000B61
:10036000000D000E000F00330034000000280000D4
:10037000000000E1001D001B0006001900050059E7
:10038000005A005B0058001100100036003700389A
:10039000000000E500010052000000E000E300E280
:1003A000002A002C00000062000000630000002A08
:1003B000000000E600E70065000000E40050005186
:1003C000004F0029003A003B003C003D003E003F4A
:1003D00000000000000000400041004200430044D3
:1003E000004500460053004A00010035001E001F72
:1003F0000020002100220023005400550056002454
:10040000002500260027002D002E002A0000004DA8
:10041000004B002B0014001A000800150017005FA5
:10042000006000610057001C0018000C001200134F
:10043000002F00300031004C004E0039000400163F
:1004400000070009000A005C005D005E0001000B6F
:10045000000D000E000F00330034000000280000E3
:10046000000000E1001D001B0006001900050059F6
:10047000005A005B005800110010003600370038A9
:10048000000000E500000052000000E000E300E290
:10049000002A002C00000062000100630001002A15
:1004A000000000E600E70065000000E40050005195
:1004B000004F0029003A003B003C003D003E003F59
:1004C00000000000000000400041004200430044E2
:1004D000004500460053004A00010035001E001F81
:1004E0000020002100220023005400550056002463
:1004F000002500260027002D002E002A0001004DB7
:10050000004B002B0014001A000800150017005FB4
:10051000006000610057001C0018000C001200135E
:10052000002F00300031004C004E0039000400164E
:1005300000070009000A005C005D005E0001000B7E
:10054000000D000E000F00330034000000280000F2
:10055000000000E1001D001B000600190005005905
:10056000005A005B005800110010003600370038B8
:10057000000000E500010052000000E000E300E29E
:10058000002A002C00000062000100630001002A24
:10059000000000E600E70065000000E400500051A4
:1005A000004F0044454255473A2064697361626CCC
:1005B00065642E0A0044454255473A20656E6162E3
:1005C0006C65642E0A0000000000000000002A2B69
:1005D00028000000000000000000000000000000F3
:1005E0000029000000002C1E34202122243426275C
:1005F000252E362D3738271E1F202122232425267D
:100600003333362E37381F0405060708090A0B0C4A
:100610000D0E0F101112131415161718191A1B1C92
:100620001D2F3130232D350405060708090A0B0C50
:100630000D0E0F101112131415161718191A1B1C72
:100640001D2F3130354C000000000000000000007C
:10065000000000000000000000000000000000009A
:10066000000000000000000000007E0F00D4FFFF2B
:10067000FFC7000000780A0025303258006C65641E
:100680005F7461736B3A20004F6E6573686F743AE4
:10069000206163746976653A2025640A000A0025A2
:1006A0003033326C62003A200025303258000A7232
:1006B0002F632030313233343536373839414243B5
:1006C0004445463031323334353637383941424388
:1006D0004445460A00290A002575002F00257500AB
:1006E0005D280025640020002564002000256400AA
:1006F00020002564007C0025303258006D6F757332
:10070000656B6579205B62746E7C78207920762039
:10071000685D287265702F61636C293A205B003137
:100720003A0964656C6179282A31306D73293A2061
:1007300025750A323A09696E74657276616C286DA6
:1007400073293A2025750A333A096D61785F737011
:100750006565643A2025750A343A0974696D655FE8
:10076000746F5F6D61783A2025750A353A097768AC
:1007700065656C5F6D61785F73706565643A2025AF
:10078000750A363A09776865656C5F74696D655FEF
:10079000746F5F6D61783A2025750A00703A0970B0
:1007A00072696E742076616C7565730A643A0973B8
:1007B00065742064656661756C74730A75703A09B6
:1007C0002B310A646E3A092D310A6C743A092B31C7
:1007D000300A72743A092D31300A4553432F713A69
:1007E00009717569740A0A7370656564203D206437
:1007F000656C7461202A206D61785F737065656433
:10080000202A2028726570656174202F2074696D1C
:10081000655F746F5F6D6178290A7768657265201E
:1008200064656C74613A20637572736F723D256400
:100830002C20776865656C3D25640A5365652068E2
:100840007474703A2F2F656E2E77696B69706564CA
:1008500069612E6F72672F77696B692F4D6F7573A2
:10086000655F6B6579730A004D3E20004D25753A32
:1008700025733E20003F0A003D2025750A003F0AEF
:100880000064656661756C74730A0025750A003F23
:100890000A000A092D2056616C756573202D0A0027
:1008A000710A000A092D204D6F7573656B657920FB
:1008B0002D0A003F00433E20004C25640A000A092F
:1008C0002D20537461747573202D0A686F73745FE3
:1008D0006B6579626F6172645F6C65647328293A35
:1008E00020253032580A6B6579626F6172645F70DF
:1008F000726F746F636F6C3A20253032580A6B65E3
:1009000079626F6172645F69646C653A2025303288
:10091000580A74696D65725F7265616433322829A3
:100920003A202530386C580A000A092D2056657285
:1009300073696F6E202D0A5649443A203078464537
:10094000454428466C656872616429205049443AE0
:100950002030783030303028646F776E6275626294
:100960006C6529205645523A203078303030310AB3
:100970004255494C443A20202846656220323720AF
:1009800032303232290A4F5054494F4E533A204C9C
:10099000554641204D4F5553454B455920455854D8
:1009A00052414B455920434F4E534F4C4520434FE6
:1009B0004D4D414E4420383139320A4743433A20A5
:1009C000352E342E30204156522D4C4942433A2088
:1009D000322E302E30204156525F415243483A2049
:1009E00061767235310A000A092D20436F6E736FEC
:1009F0006C65202D0A4553432F713A09717569744E
:100A00000A6D3A096D6F7573656B65790A000A099D
:100A10002D204D61676963202D0A443A09446562BF
:100A20007567204D65737361676520546F67676CE8
:100A3000650A583A094D6174726978204465627597
:100A400067204D6F646520546F67676C65202D20AB
:100A500053686F77206B6579707265737365732067
:100A6000696E206D617472697820677269640A4BDF
:100A70003A094B6579626F617264204465627567FB
:100A800020546F67676C65202D2053686F77206B4B
:100A900065797072657373207265706F72740A4D38
:100AA0003A094465627567204D6F75736520546F10
:100AB00067676C650A563A0956657273696F6E0A04
:100AC000533A095374617475730A433A0941637464
:100AD000697661746520436F6E736F6C65204D6F2E
:100AE00064650A46312D4631303A0953776974639B
:100AF0006820746F204C6179657220302D39202870
:100B0000463130203D204C30290A302D393A0953E6
:100B1000776974636820746F204C61796572203046
:100B20002D390A47524156453A095377697463682B
:100B300020746F204C6179657220302028616C74BC
:100B400065726E617465290A423A094A756D7020B2
:100B5000746F20426F6F746C6F616465720A4553E5
:100B6000433A094A756D7020746F20426F6F746C40
:100B70006F616465722028616C7465726E61746562
:100B8000290A453A095072696E7420454550524F02
:100B90004D2053657474696E67730A425350414324
:100BA000453A09436C65617220454550524F4D0AE4
:100BB000006B65796D61705F636F6E6669672E7239
:100BC00061773A20253032580A2E737761705F635F
:100BD0006F6E74726F6C5F636170736C6F636B3A8E
:100BE0002025750A2E636170736C6F636B5F746F81
:100BF0005F636F6E74726F6C3A2025750A2E73777F
:100C000061705F6C63746C5F6C6775693A20257501
:100C10000A2E737761705F7263746C5F72677569B7
:100C20003A2025750A2E737761705F6C616C745F72
:100C30006C6775693A2025750A2E737761705F724B
:100C4000616C745F726775693A2025750A2E6E6F44
:100C50005F6775693A2025750A2E737761705F6743
:100C6000726176655F6573633A2025750A2E737726
:100C700061705F6261636B736C6173685F62616313
:100C80006B73706163653A2025750A2E6E6B726F07
:100C90003A2025750A0064656275675F636F6E664A
:100CA00069672E7261773A20253032580A2E656EB8
:100CB00061626C653A2025750A2E6D6174726978DF
:100CC0003A2025750A2E6B6579626F6172643A204D
:100CD00025750A2E6D6F7573653A2025750A0065B6
:100CE00065636F6E6669673A0A64656661756C7400
:100CF0005F6C617965723A2025750A003F000A6DC4
:100D00006F7573653A206F66660A000A6D6F7573BA
:100D1000653A206F6E0A000A6B6579626F617264D2
:100D20003A206F66660A000A6B6579626F617264C9
:100D30003A206F6E0A000A6D61747269783A206F0A
:100D400066660A000A6D61747269783A206F6E0AED
:100D5000000A64656275673A206F66660A000A6475
:100D6000656275673A206F6E0A000A0A4A756D70EF
:100D7000696E6720746F20626F6F746C6F61646559
:100D8000722E2E2E2000433E2000436C6561726956
:100D90006E6720454550524F4D0A000A00253032FB
:100DA0005820006B6579626F6172645F7265706F65
:100DB00072743A20005B735D005B575D005B535DAE
:100DC000005B525D005B445D005B435D00160364A5
:100DD000006F0077006E0062007500620062006CB8
:100DE0000065000000100346006C0065006800729A
:100DF000006100640000000403090409025B0003B1
:100E00000100A0FA090400000103010100092111F9
:100E100001000122400007058103080001090401C7
:100E2000000103000000092111010001227B0007DD
:100E300005820320000109040200020300000009EA
:100E40002111010001222200070583032000010770
:100E50000503032000011201000200000008EDFE5E
:100E600000000100010200010631FF0974A101091F
:100E700075150026FF00952075088102097615007A
:100E800026FF00952075089102C005010902A10105
:100E900085020901A100050919012908150025018C
:100EA0009508750181020501093009311581257FF9
:100EB00095027508810609381581257F9501750809
:100EC0008106050C0A38021581257F950175088178
:100ED00006C0C005010980A101850319012AB700D8
:100EE000150126B700950175108100C0050C090198
:100EF000A101850419012AA002150126A00295016D
:100F000075108100C005010906A101050719E02936
:100F1000E715002501950875018102950175088185
:100F2000010507190029FF150026FF009506750821
:100F300081000508190129059505750191029501A2
:100F400075039101C00011241FBECFEFD0E2DEBFB8
:100F5000CDBF04B603FE18C080913B0390913C03C3
:100F6000A0913D03B0913E038730904BA740B04B1A
:100F700059F410923B0310923C0310923D031092DF
:100F80003E03E0E0F0EF099512E0A0E0B1E0ECE60E
:100F9000FBE500E00BBF02C007900D92A230B10745
:100FA000D9F723E0A2E0B2E001C01D92AB33B20753
:100FB000E1F70E941D1B0C94B42D0C940000FF93CC
:100FC000EF93E0910202F0910302309709F0099546
:100FD000EF91FF910895FC018591803011F0EFDFD2
:100FE000FBCF0895FF27E0E230E247FF0CC04195B8
:100FF00097FF09C0EDE26095709580959095611D11
:10100000711D811D911D27FF02C0219530E350E223
:10101000AA27660F771F881F991FAA1FA41710F011
:10102000A41B63955A95A9F7AA3008F0A95FA05DA3
:10103000AF93F395611571058105910541F7ED3287
:1010400011F4EF93F395F21718F43F93F395FBCF58
:101050008F91B5DFFA95E1F70895E991F9918591BE
:10106000803021F0853219F0AADFF9CF089520E011
:10107000E89455915532C1F3503311F46894559169
:101080005A3348F4505390F3220F022E220F220FAE
:10109000200D250FF4CF0EF42195899199915336A7
:1010A00019F3533729F1533559F1BC018827992792
:1010B000E8945C3621F4899199916894559154365D
:1010C00039F446EF7EF077FF0DC08FEF9FEF0AC037
:1010D00055374AE039F0583540E121F0523642E0C8
:1010E00009F00895FF93EF937DDFEF91FF91B7CF64
:1010F000FF93EF93FC0181918030B9F360DFFBCF68
:10110000FF93EF9368DFF1CFDF93CF93CDB7DEB7D7
:101110002596A3DFCF91DF910895873A2DE59207B9
:1011200021F0883A9D4541F00FC0FB018281882360
:1011300059F087ED90E006C0FB018281882321F001
:1011400084EC90E00E94560A81E0089581E00895C1
:101150000C948D0808950C94AA081F93CF93DF93E5
:1011600000D000D01F92CDB7DEB749835A836B837E
:101170003091050289819A81311114C0662359F09A
:10118000222349F00E94CA10182F682F89819A8162
:101190000E94731003C00E949E10182F69817A81EB
:1011A000812F04C00E94CA1069817A810F900F902C
:1011B0000F900F900F90DF91CF911F910C943618E4
:1011C000FC01262F408151816281738184810C94BE
:1011D000AD0881E00895CF93DF93EC0160E00E94B9
:1011E000E008BE01DF91CF910C94AB080C94B019CC
:1011F0000C94AC1908950E941D0F0E94FA082FEF5D
:1012000084E39CE0215080409040E1F700C0000062
:101210000C9476250F931F93CF93DF938C0161E09D
:101220000E94E008EC01B8010E94A808882309F494
:101230005BC0B801CE010E945323882309F454C037
:10124000B801CE010E94351E882309F44DC0B801B3
:10125000CE010E94AF22882309F446C0F8018281A2
:101260008823D9F1CF3D8CE5D80779F140F4C11539
:10127000FCE5DF0791F0C130DC4591F02EC0CC35A4
:10128000EDE5DE0741F1CD35FDE5DF0709F1CB35B1
:10129000DD4519F50E94611520C00E94FB0824C09D
:1012A0008091C502C82FC095C170C0FB80F98093A2
:1012B000C502CC2329F085EB95E00E94EB0714C012
:1012C00083EA95E00E94EB0710C00E940F160CC045
:1012D0000E94581502C00E946415C801DF91CF9189
:1012E0001F910F910C94A608C0E08C2FDF91CF9135
:1012F0001F910F9108950E94A8240C94BA0A0E948D
:10130000BD0A0C94AE24DF92EF92FF920F931F93CD
:10131000CF93DF93E82FF0E0EA53FA4FD490282FD1
:1013200026952695269530E0F901EA59F94F049162
:10133000877010E0082E02C0159507950A94E2F711
:1013400001701127F901EA5AF94FE490F12C082EA7
:1013500002C0F594E7940A94E2F791E0E922FF24B1
:10136000F901EA5BF94FC491D0E002C0D595C79569
:101370008A95E2F7C170DD270115110519F081EE9C
:101380000E94430BE114F10419F086EE0E94430B16
:101390008D2D0E94710CEF2819F086EE0E94F20B41
:1013A000012B19F081EE0E94F20BCD2B51F08CE253
:1013B000DF91CF911F910F91FF90EF90DF900C94F0
:1013C000710CDF91CF911F910F91FF90EF90DF9003
:1013D0000895EF92FF920F931F93CF93DF938C01A9
:1013E000F62E8AE0E82EF8018491882309F457C08C
:1013F000813009F042C0E8012196FE0184918130DC
:1014000031F42196FE0184910E94710C39C0823022
:1014100039F4E8012296FE0184910E94430B30C00A
:10142000833039F4E8012296FE0184910E94F20B88
:1014300027C0843029F5E8012296FE01249180E03E
:1014400090E030E0205331092A30310560F4E89E05
:10145000A001E99E500D1124C901840F951F21960A
:10146000FE012491EECF009759F0EFE9FFE03197AC
:10147000F1F700C000000197F6CF0E948309E80150
:101480008E010F5F1F4F8F2D882309F4ACCFEFE93A
:10149000FFE03197F1F700C000008150F5CFDF91F8
:1014A000CF911F910F91FF90EF90089560E00C9401
:1014B000E9098295982F937344E0949F9001112439
:1014C0008C7C86958695282B822F8575880F2A7AA5
:1014D0002695822B0895CF93DF93D92F0E94590A26
:1014E000C82F8D2F0E94590A2C2F30E0322F22272F
:1014F000A901482BCA01DF91CF910895CF92DF92C5
:10150000EF92FF920F931F93CF93DF936B017C01B8
:10151000CB010E946B0AEC01C7010E946B0AAC016F
:10152000CE01A0E0B0E0DC019927882760E070E000
:101530008C019D01042B152B262B372BC901B801DB
:10154000DF91CF911F910F91FF90EF90DF90CF909F
:10155000089508950C94A90A81E008950C94AC0AAA
:101560000895CF93C82F0E94AA0A8C2F0E94AE0A1A
:10157000CF91089580E00C94B10A0E94AF230C949F
:10158000B10ACF930E94AF23C82F80910402C817DD
:1015900041F1C09304028091C50282FF1EC080FF0A
:1015A00004C08DE796E00E94EB078091C50280FFA2
:1015B0000CC01F92CF9388E796E09F938F930E9471
:1015C00084080F900F900F900F908091C50280FFBC
:1015D00004C086E796E00E94EB078C2FCF910C9415
:1015E000B10ACF910895CF93DF93CDB7DEB72B9794
:1015F0000FB6F894DEBF0FBECDBF4F835887698703
:101600007A878B8761110E9490149E012F5F3F4F54
:1016100086E0F90111928A95E9F785E0FE01379697
:10162000D90101900D928A95E1F789819A814C81C7
:101630005D81452B31F09F3F31F491E08F3F19F4EC
:1016400003C091E001C090E090FF09C049815A8138
:101650006B817C818D819E810E94B11305C0C9017F
:101660000E94E9088111F2CF2B960FB6F894DEBFE5
:101670000FBECDBFDF91CF910895FC018081918194
:101680000E940C110895CF93882309F4A9C0C82F94
:101690008238C1F40E94AF2381FDA2C069E380912A
:1016A0000201909103010E9480240E94B2142FEF46
:1016B00081EE94E0215080409040E1F700C00000AE
:1016C00069E319C0833801F50E94AF2380FD88C00B
:1016D00063E580910201909103010E9480240E94A1
:1016E000B2142FEF81EE94E0215080409040E1F75A
:1016F00000C0000063E580910201909103010E9407
:101700008224CF910C94B2148438C1F40E94AF2388
:1017100082FD66C067E480910201909103010E94FE
:1017200080240E94B2142FEF81EE94E0215080407B
:101730009040E1F700C0000067E4DDCF8CEF8C0F34
:10174000813AF8F48C2F0E945822811149C06C2FE5
:1017500080910201909103010E944A24882349F05C
:101760006C2F80910201909103010E9482240E94BB
:10177000B2146C2F80910201909103010E94802489
:10178000C0CF80E28C0F883048F4C77081E001C080
:10179000880FCA95EAF70E947314B3CFEBE5EC0FFC
:1017A000E33040F4F0E0E95BFE4F808190E0CF91C0
:1017B0000C941224E8E5EC0FE73150F4F0E0EE0F62
:1017C000FF1FE75EFE4F80819181CF910C9428240A
:1017D000CD3E30F08C2F0E94A21BCF910C94741C34
:1017E000CF910895882309F464C0823879F40E9467
:1017F000AF2381FF5EC069E38091020190910301F4
:101800000E9480240E94B21469E310C08338B1F4AE
:101810000E94AF2380FF4DC063E58091020190914B
:1018200003010E9480240E94B21463E580910201AA
:10183000909103010E9482240C94B214843879F4AC
:101840000E94AF2382FF35C067E48091020190912E
:1018500003010E9480240E94B21467E4E7CF9CEF4A
:10186000980F913A10F4682FE1CF90E2980F9830DA
:1018700050F4877091E001C0990F8A95EAF7892F9B
:101880000E947914D9CF9BE5980F933020F480E023
:1018900090E00C94122498E5980F973120F480E0A2
:1018A00090E00C9428248D3E20F00E94FD1B0C94A7
:1018B000741C08951F93CF93DF93182FEB010E94A0
:1018C000430B209741F08FE99FE00197F1F700C0AB
:1018D00000002197F6CF812FDF91CF911F910C94BB
:1018E000F20B893319F060E070E002C060E570E04F
:1018F0000C945A0C882321F00E9473140C94B21497
:101900000895882321F00E9479140C94B21408954C
:10191000CF92DF92EF92FF920F931F93CF93DF93BB
:101920007C01D62FC72FFC011281058102950F7013
:101930000E9469148823B9F01123A9F08C2F807FAD
:10194000803421F080E28D0F883068F08091F902B8
:1019500082FD09C082E00E9412150E94691491E084
:10196000D82ED92601C0D12CCC2EC2948FE0C8220B
:101970008C2D90E08C30910508F0CFC1FC01E45B28
:10198000FF4F0C94482D8C2F807FCF70882311F04F
:10199000C295C07F112399F0CC2309F4AAC180E23B
:1019A0008D0F883010F0D11104C08C2F0E94731459
:1019B00003C08C2F0E9483140E94B2149AC18D2FF1
:1019C0000E94F20BCC2309F4A8C180E28D0F88306D
:1019D00038F1DD2329F18C2F0E94891424C08C2F2B
:1019E000807FCF70803211F0C295C07FDD2319F067
:1019F000D130A1F13DC08091F90282FF17C01123BF
:101A000049F0CC2329F08C2F0E9473140E94B21449
:101A100080E070C180E00E94F20BCC2309F47DC10C
:101A20008C2F0E9479140E94B21477C1112371F097
:101A3000002341F0013031F40E9493148C2B0E945A
:101A40009B146BC10E9493148C2B1DC0002319F0B2
:101A5000013009F462C10E94A81425C0112321F0AD
:101A6000063008F05AC10EC0053008F056C11BC040
:101A7000112361F0002331F0F701858180FF39C126
:101A80008F7085838C2F0E947A0C47C1002359F0F8
:101A9000D93309F03FC1FFEF07EE13E0F1500040EA
:101AA0001040E1F735C18C2F0E94810C36C18C2F7C
:101AB00086958695837019F0813061F02EC11123CF
:101AC00021F08D2F9C2F937002C080E090E00E9447
:101AD00012242BC1112321F08D2F9C2F937002C053
:101AE00080E090E00E94282420C18D2F112319F05E
:101AF0000E94A21B02C00E94FD1B0E94741C15C103
:101B00008C2F837009F047C011110BC12D2F229526
:101B100026952770220F220F6D2F6F70862F90E071
:101B2000A0E0B0E0022E04C0880F991FAA1FBB1FBF
:101B30000A94D2F7D4FF10C04FE050E060E070E0AC
:101B400004C0440F551F661F771F2A95D2F7409592
:101B500050956095709503C040E050E0BA01C6957D
:101B6000C695C3708A019B01082B192B2A2B3B2B8E
:101B7000C901B801C23049F058F4C13019F00E94CF
:101B8000890FCFC00E94770FCCC00E949B0FC9C0A5
:101B90000E94750FC6C0112319F08C2F817001C0EF
:101BA0008695882309F4BDC02D2F22952695277090
:101BB000220F220F6D2F6F70862F90E0A0E0B0E013
:101BC000022E04C0880F991FAA1FBB1F0A94D2F7C8
:101BD000D4FF10C04FE050E060E070E004C0440F5C
:101BE000551F661F771F2A95D2F74095509560952F
:101BF000709503C040E050E0BA01C695C695C37029
:101C00008A019B01082B192B2A2B3B2BC901B801F8
:101C1000C23049F058F4C13019F00E944E1081C012
:101C20000E943C107EC00E9460107BC00E94AF0FDB
:101C300078C0CF70112339F08C2F0E94D50F8D2FD3
:101C40000E947A0C6EC08D2F0E94810C8C2F0E94F6
:101C5000F60F67C0D23F21F128F4D03F41F0D13FC9
:101C6000C1F043C0D33F19F1D43F79F03EC01123F6
:101C700041F0053008F051C08C2F8F710E941B106D
:101C80004CC0063008F049C0F7CF8091F90282FFBE
:101C900018C0112339F08C2F8F710E94D50F3DC0D1
:101CA0001123C9F38C2F8F710E94F60F36C01123B8
:101CB00029F08C2F8F710E94C00F2FC00E94BB0F84
:101CC0002CC0112349F0CF718C2F0E94D50F63E0F7
:101CD0008C2F0E94F71421C081E00E94121502305F
:101CE000E0F082E00E94121518C0112331F00023A9
:101CF00091F28D2F0E94430B10C0002399F2D9332B
:101D000049F41FEF27EE33E0115020403040E1F757
:101D100000C000008D2F0E94F20B88EF8C0D8430E4
:101D200020F40E94AF230E94B10ADD20C9F00E9476
:101D3000651480FD15C0F70112820E945F140E9495
:101D4000D50FC7010E94D10E0E945F14DF91CF9181
:101D50001F910F91FF90EF90DF90CF900C94F60FB2
:101D6000DF91CF911F910F91FF90EF90DF90CF9077
:101D700008950F931F93CF93DF93EC0168817981CE
:101D80008A810E9417118C010E9472100E94630FB9
:101D9000B801CE010E94880CDF91CF911F910F9165
:101DA0000895CF93DF93EC01988189812B813C8149
:101DB000232B31F08F3F31F481E09F3F19F403C0B2
:101DC00081E001C080E080FD1DC0CE010E940A09B3
:101DD000811110C00E9469148823A1F08A81882390
:101DE00089F08091F90282FD0DC082E0DF91CF91F0
:101DF0000C941215CE010E94B90ECE01DF91CF9145
:101E00000C94EB08DF91CF91089580E090E00E9460
:101E1000122480E090E00E9428240E9490140E94E6
:101E2000B2140E94271E0C94741C809102019091A0
:101E300003010E9484240C94050F0E9480140C94CA
:101E4000150F92959F70963079F010F4925001C062
:101E50009A50923068F4803F69F018F4883E40F45C
:101E600009C0843F29F406C0883E20F0813F11F06C
:101E700080E0089581E00895FC01808191810E94B5
:101E80000C110E94210F0895CF93DF9300D000D052
:101E90001F92CDB7DEB70F900F900F900F900F905D
:101EA000DF91CF910895CF93DF9300D000D000D081
:101EB000CDB7DEB726960FB6F894DEBF0FBECDBF06
:101EC000DF91CF910895089508950C94640F0C94B8
:101ED000650F0E94670F60935502709356028093BE
:101EE0005702909358020C94050F0C94690F0F93AE
:101EF0001F93009155021091560220915702309184
:101F00005802602B712B822B932B1F910F910C94F5
:101F1000690F0F931F930091550210915602209163
:101F200057023091580260237123822393231F911B
:101F30000F910C94690F0F931F930091550210910C
:101F4000560220915702309158026027712782274C
:101F500093271F910F910C94690F0C94640F0E94AA
:101F6000AD0F60935102709352028093530290938D
:101F700054020C94050F60E070E0CB010C94AF0F9D
:101F80000F931F9341E050E060E070E08A019B01F5
:101F900004C0000F111F221F331F8A95D2F7C901F9
:101FA000B8011F910F910C94AF0F0F931F9341E055
:101FB00050E060E070E004C0440F551F661F771FBB
:101FC0008A95D2F78091510290915202A0915302CA
:101FD000B09154028A019B01082B192B2A2B3B2B11
:101FE000C901B8011F910F910C94AF0F0F931F936C
:101FF00041E050E060E070E004C0440F551F661FF0
:10200000771F8A95D2F7409550956095709580918D
:10201000510290915202A0915302B09154028A0150
:102020009B01082319232A233B23C901B8011F91CF
:102030000F910C94AF0F0F931F9341E050E060E0BD
:1020400070E004C0440F551F661F771F8A95D2F7B2
:102050008091510290915202A0915302B09154028A
:102060008A019B01082719272A273B27C901B801A4
:102070001F910F910C94AF0F0F931F93009151027A
:10208000109152022091530230915402602B712B17
:10209000822B932B1F910F910C94AF0F0F931F93D3
:1020A000009151021091520220915302309154023A
:1020B00060237123822393231F910F910C94AF0F00
:1020C0000F931F93009151021091520220915302DD
:1020D0003091540260277127822793271F910F9117
:1020E0000C94AF0F089524E1929F800D1124E82FE6
:1020F000E695E695E695877051E001C0550F8A9503
:10210000EAF785E0E89FF0011124EA5FFD4F20E047
:1021100030E070E04081CB01022E02C09695879599
:102120000A94E2F78170819584278523842781931F
:102130002F5F3F4F2530310569F7089524E1929FC5
:10214000800D1124682F669566956695982F977077
:1021500085E0689FB001112440E050E080E0FB0181
:10216000E40FF51FEA5FFD4F208130E0092E02C029
:10217000369527950A94E2F721703327042E01C083
:10218000220F0A94EAF7822B4F5F5F4F45305105CB
:1021900031F70895BF92CF92DF92EF92FF920F93A3
:1021A0001F93CF93DF938C01C0905102D0905202C5
:1021B000E0905302F09054028091550290915602A3
:1021C000A0915702B0915802C82AD92AEA2AFB2ABC
:1021D000CFE1D0E0D701C6010C2E04C0B695A7957B
:1021E000979587950A94D2F780FD04C0219790F7C0
:1021F000B12C07C0BC2EB8018C2F0E944918019742
:10220000A9F38B2DDF91CF911F910F91FF90EF904C
:10221000DF90CF90BF900895CF93DF93EC010E94A1
:10222000CA10BE010E944918DF91CF9108951F93F3
:10223000CF93DF93EB0190910502992321F0CB011D
:102240000E940C1113C0882349F0CB010E94CA10D0
:10225000182F682FCE010E94731004C0CB010E947A
:102260009E10182FBE01812F0E944918DF91CF9137
:102270001F9108951F93CF93DF93C091590216E0E9
:1022800080915A02C81799F0D0E01C9FF0011D9F61
:10229000F00D1124E55AFD4F408151816281738117
:1022A000848195810E94530F2196C770E9CFDF91F9
:1022B000CF911F91089540918B0250918C026091B3
:1022C0008D0270918E0280918F02909190020C94F9
:1022D000530FEF92FF920F931F93CF93DF93809151
:1022E000900282958F7009F065C080918D028823DD
:1022F00009F460C080915902F0905A0210918B024B
:1023000000918C0260918E0270918F0291E01F3FCC
:1023100009F090E0C0910001D0910101292F96E0D1
:10232000E92E8F1509F446C06115710521F00F3FA4
:1023300021F030E003C031E001C0322F90E030FDE9
:1023400036C0E89EF001E99EF00D1124DF01A55A88
:10235000BD4F11963C911197301329C03C91311318
:1023600026C012963C911297311121C013964D91BF
:102370005C911497461B570B4C175D07C0F4809176
:1023800090028F70806180939002E05AFD4F8081AF
:102390008F70806180838BE892E00E94D10EDF9184
:1023A000CF911F910F91FF90EF900C943A110196ED
:1023B0008770B7CFDF91CF911F910F91FF90EF9072
:1023C00008959F92AF92BF92CF92DF92EF92FF92C9
:1023D0000F931F93CF93DF93CDB7DEB761970FB6FF
:1023E000F894DEBF0FBECDBF8C0185E0F801DE01A1
:1023F0001D9601900D928A95E1F7D8011296EC9006
:1024000090918B02E0918C0220918E0230918F028C
:102410002115310531F0EF3F31F481E09F3F19F490
:1024200003C081E001C080E0B82FB1709B2E80FD19
:1024300047C1D8014C9111965C9111971396AD90BC
:10244000BC9014978BE8C82E82E0D82EF0908D02B5
:10245000B501621B730B2091000130910101FF2037
:1024600009F4D9C0809190026217730708F095C0F3
:10247000282F207F09F052C05E1313C0491311C0EA
:10248000FE2CE1100EC08F708061809390020E943C
:102490005B11C6010E94D10E80919002F8018583E4
:1024A0004DC1AB2831F05F3F31F481E04F3F19F46B
:1024B00003C081E001C080E080FD03C081E08E2583
:1024C00002C080E090E0F82FF170FF2E80FF1CC06A
:1024D0008091590220915A0236E0821709F40BC10B
:1024E00090E0389FF001399FF00D1124E55AFD4F1F
:1024F0006181561306C06081461303C06281E612F3
:1025000003C001968770E9CFFE2CEE2009F416C1B6
:102510008091900281608093900254C05E1306C047
:10252000491304C0E11002C0F80199C0C8010E941B
:102530003C0F882361F1EE2051F120919002822F0F
:1025400082958F7090E0029774F080918B02909149
:102550008C0298878F831986BB86AA862C87CE012A
:1025600007960E94D10E86E0F801ABE8B2E0019038
:102570000D928A95E1F70E9469110E945B110AC0D1
:102580005E1711F1C8010E943C0F81112CC0C801D7
:102590000E94D10EFF24F394D1C0282F207F81F711
:1025A0007A2DB98AA88A6E2D89890E94440F8BE8FA
:1025B00092E00E94D10E86E0D6011D928A95E9F73D
:1025C0000E945B11F12CBAC04913DCCFE110DACFC5
:1025D000F8018583C8010E94D10E86E0D6011D92C4
:1025E0008A95E9F7ABC0EE2091F220919002822FFC
:1025F00082958F7090E002970CF4B5CF80918B029A
:1026000090918C029A8389831B82BD82AC822E8337
:10261000CE010196A6CF6217730708F044C0FE2CC6
:10262000EE2009F4B4CF5E1330C049132EC02091C0
:10263000900220FD21C0822F82958F70482F50E09C
:1026400041155105C9F0F80125834F30510541F07E
:102650008F5F982F9295907F822F8F70892B858323
:10266000C8010E94D10E86E0F801ABE8B2E001900B
:102670000D928A95E1F73CC086E0F801ABE8B2E044
:1026800001900D928A95E1F759C0C8010E943C0F54
:10269000811169CF80919002816080939002C8017E
:1026A0000E94D10E4BC07A2DB98AA88A6E2D8989D5
:1026B0000E94440F86E0D6011D928A95E9F718C062
:1026C000EE2009F464CFC8010E943C0FF82E882345
:1026D00009F45DCF86E0F801ABE8B2E001900D921D
:1026E0008A95E1F78BE892E00E943D0B0E94691108
:1026F0000E945B1123C04D875E878D859E850E9459
:102700000C11292F22952F70223028F49F7039F058
:10271000811105C00BC0243028F49F7049F4805EFD
:10272000883020F0C8010E94D10E9F2CF92C06C0E1
:10273000D80115969C91907F91F7F8CF8F2D6196D7
:102740000FB6F894DEBF0FBECDBFDF91CF911F91C2
:102750000F91FF90EF90DF90CF90BF90AF909F9040
:1027600008951F93CF93DF93CDB7DEB72C970FB6A5
:10277000F894DEBF0FBECDBF4F83588769877A8735
:102780008B879C87CE0107960E94E1118823D1F0A8
:102790009F8188852A853B85232B31F08F3F31F43B
:1027A00081E09F3F19F403C081E001C080E080FD1B
:1027B00047C04F81588569857A858B859C850E94A5
:1027C000530F3EC086E0FE013796DE011196019060
:1027D0000D928A95E1F7FF81E8856A857B85611511
:1027E000710531F0EF3F31F481E0FF3F19F403C090
:1027F00081E001C080E080FD23C020915A0230E0DA
:10280000C9010196877099274091590250E08417B9
:102810009507F1F1F983EA837D836C8396E0929FBB
:10282000D001939FB00D1124A55ABD4FFE013196E2
:1028300001900D929A95E1F780935A020E943A1105
:1028400016E08091590290915A02891771F1189FF0
:10285000C0011124855A9D4F0E94E111882329F15E
:10286000E09159021E9FF0011124E55AFD4F40816D
:10287000518162817381848195810E94530F80917F
:10288000590290E001968770992780935902D9CF19
:102890000E941D0F10925A0210925902EBE8F2E0CA
:1028A00086E0DF011D928A95E9F72C960FB6F89421
:1028B000DEBF0FBECDBFDF91CF911F9108958091F4
:1028C00099028595859585950895809199028770DF
:1028D000089590919902977081E009F480E008953D
:1028E0008091A40208959091A402892B8093A40260
:1028F000089580959091A40289238093A40208955D
:102900001092A40208959091A302892B8093A302B0
:10291000089580959091A30289238093A30208953E
:102920001092A302089580919A02089508950C943C
:1029300096140C9497149091F90292FD08C090910E
:102940009A02981721F080939A020C949914089592
:1029500080919A02882329F010929A0280E00C94C8
:1029600099140895CF93DF93E0910201F091030150
:102970008091A4028083E0910201F0910301908193
:102980008091A302892B808380919A02882381F011
:10299000E0910201F09103019081892B8083809165
:1029A0000201909103010E943E2481110E94A8140B
:1029B000C0910201D091030148E050E061E972E06A
:1029C000CE010E94652D892B69F088E0FE01A1E906
:1029D000B2E001900D928A95E1F7CE01DF91CF919F
:1029E0000C94BB23DF91CF9108950C949614909191
:1029F000F90292FD10C098E0899F90011124262BC6
:102A0000209399020E94D50F809199028595859512
:102A100085950C94F5140C94D50F1092990280E0D2
:102A20000C94F51420919902809582238093990249
:102A3000982F977099F430E0482F082E000C550B12
:102A40002417350759F09091F90292FD07C085953A
:102A5000859585950E94F60F0C940D150895CF93DA
:102A60009091F90292FB222720F92817F9F0C82F3C
:102A7000892FC0FB82F98093F9028091F80290912E
:102A8000F9020E948B1582E00E9412158091C50206
:102A900080FF0CC01F92CF9388E896E09F938F939E
:102AA0000E9484080F900F900F900F90CF9108957F
:102AB0008091F90282FB882780F991E089270C94A4
:102AC0002F1581E00C942F1580E00C942F1580E0D9
:102AD00090E00E947A2D21E0893E9E4F09F020E08F
:102AE000822F089582E090E00C94722D83E090E0B4
:102AF0000C94722DCF9384E090E00E94722DC82F29
:102B000082E290E00E94722D2C2F30E0A901582B18
:102B1000CA01CF910895CF93C92F682F84E090E028
:102B20000E94802D6C2F82E290E0CF910C94802D3A
:102B3000AB01BC018FE090E00C94922DAB01BC0185
:102B400083E190E00C94922D60E070E0CB010C9456
:102B50009E1560E070E0CB010E9498150C94A415BE
:102B600069EE7EEF80E090E00E949E2D60E082E0C2
:102B700090E00E94802D60E083E090E00E94802D34
:102B8000109255021092560210925702109258025B
:102B900060E084E090E00E94802D60E082E290E0BE
:102BA0000E94802D60E085E090E00E94802D60E032
:102BB00086E090E00E94802D6FEF87E090E00E9419
:102BC000802D40E050E0BA0188E090E00E94922D14
:102BD00060E08DE090E00E94802D40E050E0BA017E
:102BE00088E190E00E94922D60E087E190E00E94F1
:102BF000802D40E050E0BA018CE190E00E94922DDF
:102C000060E070E080E290E00E949E2D40E050E0A5
:102C1000BA0188E190E00E94922D0C94A9150C94C1
:102C2000B015682F8EE090E00C94802D0E94352521
:102C30006093C1027093C2028093C3029093C40256
:102C40006093BD027093BE028093BF029093C00256
:102C5000089585B7806885BF85B7806885BF08956A
:102C600081E008950C94301608950C9434160C9459
:102C700034160C9437160C9434160C943B160C94A2
:102C800034160E9429168BE697E20E94A5230E9423
:102C90003F160C943D160E9435160C9434160E9473
:102CA00026190C94B00A0E9420250E94741A0E94D2
:102CB0004F160C9439162F923F924F925F926F925B
:102CC0007F928F929F92AF92BF92CF92DF92EF92BC
:102CD000FF920F931F93CF93DF93CDB7DEB72D975E
:102CE0000FB6F894DEBF0FBECDBF0E94891A282E02
:102CF00081110E94161685EA92E09D878C8700E07C
:102D000010E0302E802F0E944A192B013C01EC85E7
:102D1000FD8581919191A191B191FD87EC8753013E
:102D2000420188269926AA26BB2681149104A10473
:102D3000B104B1F40F5F1F4F0630110511F78FEF8B
:102D400089838A831B820E9429258160782F9D8335
:102D50008C8349815A816B818D810E94F30A51C015
:102D60008091C50281FD0E9456191B86C12CD12C71
:102D70007601C394D501C4018C219D21AE21BF21D0
:102D8000892B8A2B8B2B91F10E9432168823D1F04C
:102D9000FB85FE833F824C205D206E207F2081E0FA
:102DA00045284628472809F480E088870E9429257D
:102DB0008160782F9A8789874E815F8168858A85AF
:102DC0000E94F30A000F111F000F111FF801EB55AD
:102DD000FD4F80819181A281B381C826D926EA2640
:102DE000FB26C082D182E282F3820BC08B858F5F8B
:102DF0008B87CC0CDD1CEE1CFF1C843109F0BACF94
:102E000099CF81E0211001C080E02D960FB6F89493
:102E1000DEBF0FBECDBFDF91CF911F910F91FF900D
:102E2000EF90DF90CF90BF90AF909F908F907F906A
:102E30006F905F904F903F902F9008950E945B1687
:102E40000E94141D0C94C10ACF93DF930E944E1868
:102E5000EC01811521E5920708F045C0811530E5A8
:102E6000930708F094C0883E910528F5803E9105AF
:102E700008F0F8C0883A910570F4853A910508F099
:102E80007CC08130910509F475C008F4E8C004974E
:102E900008F0E8C0E4C08F3B910508F0E0C0C85AD4
:102EA000D0E0CC0FDD1FC65BDE4F0990D881C02D6E
:102EB000CE019464D8C0811540E2940758F481157E
:102EC00051E0950708F0CEC08D3E910508F4C7C0CB
:102ED0009065C9C0C11580E4D80708F4C0C0DF7090
:102EE000CE01906AC0C0811525E59207A8F481152E
:102EF00034E5930708F095C0811543E5940708F081
:102F00007BC0811552E5950708F061C0D82FCC270A
:102F1000CE01816F906AA7C0C11589E5D807A0F4DA
:102F2000C11528E5D20708F082C0C11536E5D307E0
:102F300008F095C08C2F0E94E2188F7190E0D82F76
:102F4000CC27CE0190628FC0C1154AE5D40708F4A2
:102F500074C0CE0190568115904208F080C08D2F2C
:102F60008F710E94E218DD27D0628F71AE01582B5D
:102F7000CA0179C081E090E076C0C55AD0E0C85857
:102F8000DE4F8881C82FD0E0CE0190646CC074E021
:102F9000969587957A95E1F7282F23703C2F33700B
:102FA00081E090E002C0880F991F3A95E2F79C6893
:102FB000AC01522B9A019C2F9F709695969550E2EA
:102FC000959FE0011124C9018C2B9D2B4CC083706F
:102FD000992721E030E002C0220F331F8A95E2F7E3
:102FE0009C2F9695969580E2989FE0011124C22B24
:102FF000D32BCE019C6837C08370992721E030E045
:1030000002C0220F331F8A95E2F79C2F9695969562
:1030100040E2949FE0011124C22BD32BCE019A6889
:1030200022C0D82FCC27CE01846F906A1CC0DC2F21
:10303000CC27CE01806F906A16C08C2F8F700E94B3
:10304000E21894E0D695C7959A95E1F7CF70D0E055
:10305000DC2FCC27D0699E01282BC90104C080E059
:1030600090E001C0CE01DF91CF91089528E7829FC3
:10307000C0011124FC0124E1729FE00DF11D112417
:10308000E60FF11DEE0FFF1FED50FF4F859194915C
:1030900008950E9436180E942417089582389105D9
:1030A00069F1B0F48133910509F46DC048F48932B7
:1030B000910509F463C08A32910509F469C0089545
:1030C0008533910509F455C089339105B9F0089508
:1030D000833E910569F138F4803E9105B1F0823E5E
:1030E000910509F10895863E9105A9F1873E910564
:1030F000B9F1843E910509F064C023C02091F80223
:1031000020FD4FC021FD4DC008958091F80280FD43
:1031100044C08091F90280FF44C08091F80284FD90
:1031200042C083EE4DC08091F80282FF38C0F5CFD7
:103130008091F80282FD33C08091F90280FD31C098
:10314000ECCF8091F90281FF32C08091F80284FDBA
:103150002AC087EE35C08091F80283FF26C0F5CFE4
:103160008091F80283FD21C08091F90281FD1FC08A
:10317000ECCF8091F80285FD1CC01DC08091F80243
:1031800085FD19C016C08091F80286FD16C017C0D3
:103190008091F80286FD13C010C089E311C082EE51
:1031A0000FC080EE0DC080E00BC086EE09C084EE3B
:1031B00007C089E205C085E303C08AE201C081E35C
:1031C00090E008959091F80292FF0DC0282F287189
:1031D000283019F4877F846006C0282F247124309A
:1031E00011F48B7F886093FF0DC0282F2871283140
:1031F00019F4877E846106C0282F2471243111F4CC
:103200008B7E88612091F90220FF0DC0382F387124
:10321000383019F4877F816006C0382F3171313022
:1032200011F48E7F886021FF0DC0282F287128316E
:1032300019F4877E816106C0282F2171213111F494
:103240008E7E886194FD877E089508950E9467159B
:10325000811102C00E940F160E9472158093C50250
:103260000E947A159093F9028093F8020E94251922
:103270000E947615682F70E080E090E00E94750F44
:1032800060915102709152028091530290915402C8
:103290000C94AD0F24E0829FC0011124FC01EE5E6E
:1032A000FC4F60817181828193810895CF92DF927A
:1032B000EF92FF920F931F93CF93DF938EEA96E0E6
:1032C0000E94EB0782E1E82E83E0F82EC0E0D0E018
:1032D00099EAC92E96E0D92E0FE916E0DF93CF9335
:1032E000DF92CF920E94840886EA96E00E94EB0764
:1032F000F70161917191819191917F010E947E0A04
:103300009F938F937F936F931F930F930E948408D3
:103310008DE996E00E94EB0721968DB79EB70A963D
:103320000FB6F8949EBF0FBE8DBFC630D105B1F663
:10333000DF91CF911F910F91FF90EF90DF90CF9091
:10334000089580EA8A95F1F7089500C008950C94D5
:10335000A11908950C94A9190C94AA190C94A919EF
:103360000C94AE19F894E82FE295EF70F0E031A1DB
:10337000282F2F7081E090E001C0880F2A95EAF78E
:10338000982F9095932391A392A1892B82A378944F
:1033900008950F931F93CF93DF93CFE8D1E08991E6
:1033A0008F3F11F00E94B21981E0C539D807B9F7F3
:1033B000CBE7D1E00FE811E089918F3F11F00E9437
:1033C000B2190C171D07C1F7DF91CF911F910F9113
:1033D00008954F925F926F927F928F929F92AF92D9
:1033E000BF92DF92EF92FF920F931F93CF93DF93E1
:1033F0008C01C62FD0E0CE0181579E4F7C01FC018D
:1034000090819F3F09F460C0D62EF894E92FE29591
:10341000EF70F0E081A19F7021E030E001C0220F49
:103420009A95EAF7822B81A382A12095282322A3D3
:1034300078940E94A519EBE7F1E02FE831E0412CE8
:10344000512C32014394812C912C540181918F3F56
:1034500099F0A82FA295AF70B0E090964C9150E0F3
:103460008F70BA0102C0759567958A95E2F760FD85
:1034700003C0D301C20103C080E090E0DC01882AD0
:10348000992AAA2ABB2A440C551C661C771C2E17A5
:103490003F07E1F6F70180818F3F11F00E94B219DA
:1034A00061E081149104A104B10409F460E08D2D60
:1034B0000E94A719CC0FDD1FCC0FDD1FC00FD11F3D
:1034C00088829982AA82BB82DF91CF911F910F914E
:1034D000FF90EF90DF90BF90AF909F908F907F9084
:1034E0006F905F904F9008950E94C91988E1E2E1C2
:1034F000F3E0DF01982F1D929A95E9F7EAEFF2E0E9
:10350000DF011D928A95E9F786E00E94D41A0C9497
:10351000F608FF920F931F93CF93DF93CDB7DEB7DB
:1035200068970FB6F894DEBF0FBECDBF8E010F5F58
:103530001F4F88E1F80111928A95E9F7F12C6F2D60
:10354000C8010E94E919F394F6E0FF12F8CF48E1B0
:1035500050E0B8018AEF92E00E94652DFF24F394B9
:10356000009709F4F12C892B41F088E1F801AAEFCA
:10357000B2E001900D928A95E1F72F2D46E062E1CD
:1035800073E08AEF92E00E94D51A0E94F8088F2D0E
:1035900068960FB6F894DEBF0FBECDBFDF91CF9116
:1035A0001F910F91FF9008950895FF920F931F931D
:1035B000CF93DF93F82ED92F8B01C42F222349F00C
:1035C00081E08093C8020E9429259093C7028093CE
:1035D000C6028091C8028823F1F08091C6029091C2
:1035E000C7020E9441250597B0F0EF2DFD2FD801AD
:1035F00080E090E04C2F50E08417950754F401913F
:103600001191219131910D931D932D933D9301962D
:10361000F3CF1092C802DF91CF911F910F91FF90CD
:1036200008950E94E7270E9453160C94F3270E94E6
:10363000F7270E941E170C9415280E94C7240E9489
:10364000CE270E9441160E94111B0E94171B0E9448
:103650004B16FBCF8091CF0280FF06C0609109011D
:1036600070E0660F771F26C081FF04C060910901DA
:1036700084E005C082FF07C06091090188E0689F6F
:10368000B001112417C09091CE029923D1F060911E
:103690000801961788F72091090188E0289F90017A
:1036A0001124929FA001939F500D112470E0CA0134
:1036B0000E94342D6038710540F46115710519F4CC
:1036C00006C068E070E0862F08958FE7089581E0D6
:1036D00008958091CF0280FF08C06091050170E0DD
:1036E000759567957595679521C081FF06C06091B6
:1036F000050170E07595679519C082FF04C060915F
:10370000050170E010C09091CD02992399F060916D
:1037100004019617A0F780910501899FC00111242B
:1037200070E00E94342D6038710540F46115710518
:1037300019F406C061E070E0862F08958FE70895C0
:1037400081E008958D3E21F40E942A1B819504C0DA
:103750008E3E29F40E942A1B8093D30208958F3E47
:1037600021F40E942A1B819504C0803F29F40E9405
:103770002A1B8093D2020895893F19F40E94691B85
:1037800005C08A3F31F40E94691B81958093D40261
:1037900008958B3F21F40E94691B819504C08C3FE2
:1037A00029F40E94691B8093D50208959FE0980F29
:1037B000983078F421E030E0A90102C0440F551F91
:1037C0009A95E2F7CA019091D102892B8093D10298
:1037D00008958D3F21F48091CF0281600BC08E3F10
:1037E00021F48091CF02826005C08F3F29F480913F
:1037F000CF0284608093CF0208958D3E39F490917A
:10380000D30297FF35C01092D30259C08E3E29F4DF
:103810009091D3021916BCF32BC09091D2028F3E27
:1038200029F497FF25C01092D20249C0803F19F4B5
:103830001916CCF31DC09091D402893F29F41916B2
:10384000BCF41092D4023BC08A3F19F497FF10C019
:10385000F8CF8B3F39F49091D50297FF09C01092B1
:10386000D5022DC08C3F21F49091D5021916BCF3DE
:103870009FE0980F983080F421E030E0A90102C069
:10388000440F551F9A95E2F7CA0180959091D10295
:1038900089238093D10213C08D3F21F48091CF0200
:1038A0008E7F0BC08E3F21F48091CF028D7F05C0AB
:1038B0008F3F29F48091CF028B7F8093CF0280913C
:1038C000D202811106C08091D302811102C01092F0
:1038D000CE028091D402811106C08091D50281115F
:1038E00002C01092CD0208958091C50283FF7EC070
:1038F0008CEF96E00E94EB078091D1021F928F938C
:1039000087EF96E09F938F930E94840885EF96E05F
:103910000E94EB078091D202282F082E000C330B57
:103920003F938F9382EF96E09F938F930E9484083A
:1039300080EF96E00E94EB078091D302282F082E9B
:10394000000C330B3F938F938DEE96E09F938F93F4
:103950000E9484088BEE96E00E94EB078091D402CF
:10396000282F082E000C330B3F938F9388EE96E0A0
:103970009F938F930E94840886EE96E00E94EB0747
:103980008091D502282F082E000C330B3F938F9384
:1039900083EE96E09F938F930E94840880EE96E0DA
:1039A0000E94EB078091CE021F928F938DED96E0DF
:1039B0009F938F930E9484088BED96E00E94EB0703
:1039C0008091CF021F928F9388ED96E09F938F9303
:1039D0000E94840885ED96E00E94EB078DB79EB7A4
:1039E0004C960FB6F8949EBF0FBE8DBF0E9429253E
:1039F0002091D202211104C02091D302222321F070
:103A00009093CC028093CB022091D402211104C068
:103A10002091D502222321F09093CA028093C902FB
:103A200080ED92E00C940424EF92FF920F931F9389
:103A3000CF93DF9300D000D000D0CDB7DEB786E0C3
:103A4000E0EDF2E0DE01119601900D928A95E1F72A
:103A5000E090D202F090D3020091D4021091D502EE
:103A60001092D2021092D3021092D4021092D50278
:103A7000E11003C0FF2009F45DC08091CB0290915A
:103A8000CC020E944125AC019091CE02992339F0DD
:103A900020910A0130E02417350758F04BC02091DF
:103AA0000B018AE0289F900111242417350718F094
:103AB00041C09F3F19F09F5F9093CE02EE2061F0CE
:103AC0000E942A1B1E1414F09FEF01C091E0989FE2
:103AD000902D11249093D202FF2061F00E942A1BA6
:103AE0001F1414F09FEF01C091E0989F902D1124B6
:103AF0009093D3023091D2023323E1F02091D3028C
:103B00002223C1F045EB3403C0011124992319F09D
:103B10009093D20203C081E08093D20235EB23035D
:103B2000C0011124992319F09093D30203C081E0BE
:103B30008093D302011103C0112309F45DC0809169
:103B4000C9029091CA020E944125AC019091CD0218
:103B5000992339F02091060130E02417350758F0F9
:103B60004BC0209107018AE0289F9001112424175F
:103B7000350718F041C09F3F19F09F5F9093CD0229
:103B8000002361F00E94691B101614F09FEF01C022
:103B900091E0989F902D11249093D402112361F00D
:103BA0000E94691B111614F09FEF01C091E0989FCD
:103BB000902D11249093D5023091D4023323E1F05B
:103BC0002091D5022223C1F045EB3403C00111241A
:103BD000992319F09093D40203C081E08093D4021A
:103BE00035EB2303C0011124992319F09093D502DA
:103BF00003C081E08093D5028091D20281110BC075
:103C00008091D302811107C08091D402811103C039
:103C10008091D50281110E94741CEB82FC820D837D
:103C20001E8386E0FE013196A0EDB2E001900D9278
:103C30008A95E1F726960FB6F894DEBF0FBECDBF8A
:103C4000DF91CF911F910F91FF90EF900895E0EDDC
:103C5000F2E086E0DF011D928A95E9F71092CE022C
:103C60001092CD021092CF020895CF93DF93EC0112
:103C7000FB018281882309F43CC1C430FDE5DF07E4
:103C800060F4CB3F9CE5D90788F49E0122503C4567
:103C90002431310508F02EC109C0C236EDE5DE073A
:103CA00029F0C63AFDE5DF0709F024C10E947A1524
:103CB0009093F9028093F802C1318CE5D80709F49A
:103CC000C6C008F042C0C930ECE5DE0709F49BC06D
:103CD00000F5C5308CE5D80709F485C078F4C33009
:103CE000ECE5DE0709F478C008F07AC0C230DC45A4
:103CF00009F0F5C08091F8028160EFC0C7309CE503
:103D0000D90709F478C008F07AC08091F802806180
:103D1000E4C0CD30FCE5DF0709F487C058F4CB30B0
:103D20009CE5D90709F479C008F07BC08091F802BE
:103D300088606FC0CF30FCE5DF0709F480C008F071
:103D400082C08091F802877FC8C0CE3F9CE5D9072A
:103D500009F471C000F5C531FCE5DF0709F485C041
:103D600068F4C3319CE5D90709F475C008F095C023
:103D70000E941D0F8091F8028F77AFC0CC3FFCE509
:103D8000DF07A9F108F054C0CB3FDC4509F0A7C01C
:103D90008091F90240C0C230EDE5DE0709F489C028
:103DA00058F4C1158DE5D80709F45AC008F069C068
:103DB0008091F90282602FC0C236EDE5DE0709F47A
:103DC0007CC0C63AFDE5DF0709F481C0C330DD459C
:103DD00009F085C080E06EC08091F80282607DC0ED
:103DE0008091F80216C08091F802886076C08091B8
:103DF000F90282604FC08091F80280626EC08091AB
:103E0000F80280646AC00E941D0F8091F8028068E9
:103E100064C0846062C081603DC08091F8028E7F82
:103E20005CC08091F8028D7F58C08091F80216C066
:103E30008091F90218C08091F9028D7F2BC080918A
:103E4000F8028F7E4AC08091F8028F7D46C0809133
:103E5000F8028F7B42C08091F802877F8B7F3DC044
:103E60008091F9028D7F8E7F15C08091F80282FBD0
:103E7000222720F991E0922790FB82F990FB83F9A9
:103E80002CC08091F902982F909591708E7F892B8C
:103E900090FB81F98093F90222C00E941D0F80914E
:103EA000F80287FB222720F991E0922790FB87F9FF
:103EB00014C081E00E94111612C08091F80284FBA8
:103EC000222720F991E0922790FB84F906C0809187
:103ED000F802982F909590FB80F98093F8028091DA
:103EE000F8029091F9020E948B150E941D0F80E04C
:103EF00001C081E0DF91CF910895809104011F926C
:103F00008F93809105011F928F93809108011F92DA
:103F10008F93809109011F928F9380910A011F92C4
:103F20008F9380910B011F928F938FE197E09F9366
:103F30008F930E9484088DB79EB70E960FB6F894A3
:103F40009EBF0FBE8DBF0895883220F58E3108F0D8
:103F500068C08B3091F1C0F4873009F0BEC081E0B9
:103F600080930B0184E180930A018AE08093090128
:103F70008EE18093080188E08093050188E28093B8
:103F8000040181E898E0C6C0833109F443C084315C
:103F900069F1A3C08F3409F49EC028F4893231F14D
:103FA000883359F09AC0813531F008F4D4C0823595
:103FB00009F4A7C092C08FEFA5C083EA98E00E94E1
:103FC000EB070E947D1F1F9281E08F931F9288E074
:103FD0008F938CE997E09F938F930E9484080F90B2
:103FE0000F900F900F900F900F9096C080EA98E07E
:103FF0000E94EB078091DA02882309F4AAC010928C
:10400000DA021092D9021092D8021092D7021092BE
:10401000D602B1C082E998E00E94EB070E947D1FA2
:104020007BC08D518093DA02833031F170F481309E
:10403000D1F0823009F03FC08AE091E09093D9023C
:104040008093D80282EA91E01FC0853059F108F1CF
:10405000863089F584E091E09093D9028093D8026C
:104060008DED91E011C08BE091E09093D9028093A7
:10407000D80289E991E008C089E091E09093D902E3
:104080008093D8028EEA91E09093D7028093D60273
:1040900018C088E091E09093D9028093D8028BEB0E
:1040A00091E0F2CF85E091E09093D9028093D8021D
:1040B0008AEC91E0E9CF1092DA028FE898E00E9452
:1040C000EB078091DA02882309F455C01F928F9381
:1040D0008BE898E00DC08AE015C08EE798E01AC022
:1040E00097FF47C0108280811F928F9388E798E0E6
:1040F0009F938F930E9484080F900F900F900F90C2
:104100000BC081E0E091D802F091D902309729F5F7
:1041100085E798E00E94EB072091DA02222359F10B
:104120008091D6029091D702009711F485E991E031
:104130009F938F931F922F938CE698E09F938F937A
:104140000E9484080F900F900F900F900F900F9087
:1041500016C080E0089586EFD5CF2081082E000C90
:10416000990B820F911D8F3F910509F00CF4B8CF88
:104170008FEF8083B8CF88E698E00E94EB0781E05C
:104180000895CF93C82F1F928F9389EB98E09F9348
:104190008F930E94840881E090E0A0E0B0E0BC0131
:1041A000CD0104C0660F771F881F991FCA95D2F7EB
:1041B0000E94750F0F900F900F900F90CF910C945D
:1041C0001D0FEF92FF920F931F93CF93DF938B31CD
:1041D00009F4EDC008F08EC08B3009F4B1C008F0CE
:1041E00078C0863009F4AFC020F4853009F4BDC032
:1041F0004EC1873009F4C0C0883009F048C10E9420
:1042000076151F928F938FED9CE09F938F930E9462
:1042100084080E94721583FB992790F91F929F933F
:1042200082FB992790F91F929F9381FB992790F920
:104230001F929F93982F91701F929F931F928F931D
:1042400086E99CE09F938F930E9484080E947A15D0
:1042500087FB222720F91F922F9386FB222720F924
:104260001F922F9385FB222720F91F922F9384FB07
:10427000222720F91F922F9383FB222720F91F92D8
:104280002F9382FB222720F91F922F9391FB222745
:1042900020F91F922F93292F21701F922F9381FBBA
:1042A000222720F91F922F93282F21701F922F93DE
:1042B0009F938F9381EB9BE09F938F930E94840841
:1042C0008DB79EB788960FB6F8949EBF0FBE8DBF70
:1042D00035C0803109F495C020F48E3009F47BC0DC
:1042E000D6C0863109F4A8C0893109F0D0C089E26E
:1042F00099E084C08A32E1F060F4873209F4C3C0E7
:1043000028F48E3108F4C3C08D51BEC0893269F1E2
:10431000BEC0833448F48A3308F0B3C0853309F44F
:10432000B2C0883369F0B3C0833409F4ACC0AFC005
:104330008AE89DE00E94EB070E940F16C1E0ACC026
:104340008EE09AE05BC08091C502817F8E7F809372
:10435000C50287EE99E00E94EB0786E89DE00E9487
:10436000EB0781E08093DB02E9CF8AE69DE00E94C3
:10437000EB070E94FB08E2CF8091C502C82FC095D1
:10438000C170C0FB80F98093C502CC2329F08EE573
:104390009DE00E94EB0780C081E59DE00E94EB0755
:1043A0008091C502897F877F8093C502C7CF909196
:1043B000C50291FBCC27C0F981E0C827892FC0FB3B
:1043C00081F98093C502CC2319F084E49DE029C0D3
:1043D00086E39DE013C09091C50292FBCC27C0F903
:1043E00081E0C827892FC0FB82F98093C502CC23C6
:1043F00019F087E29DE015C087E19DE00E94EB0780
:104400009DCF9091C50293FBCC27C0F981E0C827CE
:10441000892FC0FB83F98093C502CC2351F08BE038
:104420009DE00E94EB078091C50281608093C502E8
:1044300033C08EEF9CE0E2CF0E943525162F072F68
:10444000F82EE92ED091F702C09118010E94AF23F7
:10445000EF92FF920F931F931F92DF931F92CF93C0
:104460001F928F938EEB98E09F938F930E94840806
:104470008DB79EB70C960FB6F8949EBF0FBE8DBF3A
:104480005DCF895301C080E00E94C12057CF8CEFDF
:104490009CE00E94EB07C0E08C2FDF91CF911F9131
:1044A0000F91FF90EF90089580E008950C945422AE
:1044B000CF93C82F8091DB02813071F040F08230C1
:1044C00009F045C08C2F0E94A41F81E046C00E94C5
:1044D00070148232F1F504C00E947014823261F4CB
:1044E0008C2F0E945622811104C08C2F0E94E12043
:1044F0002CC081E090E029C08C2F0E9454228111B1
:1045000023C0C431C9F058F4CB3069F0C031B9F4DC
:1045100082E08093DB0288E30E94A41F15C0C932A9
:1045200059F0C83361F487EE99E00E94EB0785EB00
:1045300098E00E94EB0708C01092DB020CC083EBEE
:1045400098E00E94EB0707C081E0817006C01092DE
:10455000DB0280E002C080E0F8CFCF910895CF93D6
:10456000DF9386319C4541F5EB010E947014982F32
:104570008A812091020130910301882379F09A7A8F
:1045800081E009F480E08093DC02911102C069E2CD
:1045900001C065E3C9010E9480240AC08091DC0249
:1045A000811102C069E201C065E3C9010E94822451
:1045B0000E94B21480E001C081E0DF91CF910895A4
:1045C0000F931F93CF93DF93C42FD22FFC018281CF
:1045D0008823C9F04093DF020E9429259093DE02D0
:1045E0008093DD0280E28C0F883008F057C0C770DE
:1045F00081E001C0880FCA95EAF7DF91CF911F9142
:104600000F910C947A0C8091DF02481330C0809196
:10461000DD029091DE020E944125883C910538F52B
:1046200010E21D0FCD17B9F080E28C0F883040F4F6
:10463000C77081E001C0880FCA95EAF70E94810C1B
:10464000183028F581E09D2F977001C0880F9A954A
:10465000EAF70E947A0C802F0E94710C1830F0F457
:10466000D77081E001C0880FDA95EAF70AC080E2CE
:104670008C0F883098F4C77081E001C0880FCA950C
:10468000EAF7DF91CF911F910F910C94810C802F4D
:10469000DF91CF911F910F910C94710CDF91CF910D
:1046A0001F910F9108950F939C01CB01243F4CE57E
:1046B000340731F188F4293DFCE53F07D9F02A3D64
:1046C0004CE5340779F1283D3C45A9F506E221EE99
:1046D00041EE68ED7CE52BC0263FFCE53F07E1F0AD
:1046E000A8F0273F3C4539F507E225EE46EE67EF97
:1046F0007CE51DC007E225EE45EE69ED7CE517C0BF
:1047000006E221EE40EE64EF7CE511C007E225EE03
:1047100044EE65EF7CE50BC006E221EE42EE66EF6B
:104720007CE505C008E221E045EE6AED7CE50E94EB
:10473000E02280E008C0FC018281882319F01092F9
:10474000DF0201C081E00F910895909303028093EE
:10475000020208959093E5028093E4020895E091A7
:10476000E402F091E502309721F00190F081E02D14
:10477000099480E00895EF92FF920F931F93CF93D7
:10478000DF93E091E402F091E5023097B1F18C0102
:104790000280F381E02D09958091C50282FF2DC032
:1047A00080FF04C083EA9DE00E94EB07E80118E067
:1047B0008DE9E82E8DE0F82E8091C50280FF0BC0B8
:1047C00088811F928F93FF92EF920E9484080F902E
:1047D0000F900F900F90115021961111EDCF8091F5
:1047E000C50280FF0AC08BE99DE0DF91CF911F9148
:1047F0000F91FF90EF900C94EB07DF91CF911F91F9
:104800000F91FF90EF900895E091E402F091E5029E
:10481000309739F022E0DC012C930480F581E02D03
:10482000099408952091E2023091E3022817390794
:1048300071F09093E3028093E202E091E402F09140
:10484000E502309721F00680F781E02D0994089564
:104850002091E0023091E1022817390771F090931E
:10486000E1028093E002E091E402F091E5023097EA
:1048700021F00084F185E02D09940895FC01329621
:1048800097E080E0915029F021912223D9F38F5FA6
:10489000F9CF0895662349F0FC01329608962191DC
:1048A000621729F0E817F907D1F780E0089581E051
:1048B00008959C01FC0132969FEF80E041914617DC
:1048C00089F09F3F19F4411101C0982F8F5F863006
:1048D000A9F79F3F39F0F901E90FF11D97FDFA950E
:1048E0006283089508959C012A5F3F4FFC01428135
:1048F000461301C01282019682179307B9F70895F3
:104900000C9459240C947324029626E0FC01119215
:104910002A95E9F7089508950C948B2483E08093F9
:10492000E6020C948C24811102C081E001C082E077
:104930008093E6020C948C240C94932481E0809361
:10494000E6020C948C240C949E2408950C94A524C7
:104950000C94A6240C94A5240C94A5240C94A524B2
:10496000CF930E94AC240E94891A0E94AA24C0E01E
:104970008C2F0E944A19672B682B692B29F4CF5F73
:10498000C630B1F780E001C081E0CF91089508956D
:104990001F920F920FB60F9211248F939F93AF9394
:1049A000BF938091E702811113C080912A039091F7
:1049B0002B03A0912C03B0912D034196A11DB11D95
:1049C00080932A0390932B03A0932C03B0932D0381
:1049D000BF91AF919F918F910F900FBE0F901F903D
:1049E000189580913203843031F10E947B09109236
:1049F000E70220E488E190E00FB6F894A895809350
:104A000060000FBE2093600083B7817F846083BF06
:104A100083B7816083BF7894889583B78E7F83BF87
:104A20000FB6F894A895809160008861809360002B
:104A3000109260000FBE08950E941D0F0C947F0914
:104A400082E084BD93E095BD9AEF97BD80936E00A0
:104A500008952FB7F89480912A0390912B03A09189
:104A60002C03B0912D032FBF08952FB7F8946091B8
:104A70002A0370912B0380912C0390912D032FBF5B
:104A800008959C014FB7F89480912A0390912B03CD
:104A9000A0912C03B0912D034FBF821B930B08955F
:104AA00078941F920F920FB60F9211248F939F93B9
:104AB000AF93BF9380912A0390912B03A0912C0375
:104AC000B0912D030196A11DB11D80932A039093EF
:104AD0002B03A0932C03B0932D03BF91AF919F9113
:104AE0008F910F900FBE0F901F90189581E08093CB
:104AF000E00080E28093D8001092C9008FE19EE42C
:104B00000197F1F700C0000087E090EBDC01809393
:104B10003B0390933C03A0933D03B0933E039CE082
:104B200088E10FB6F894A895809360000FBE90932B
:104B30006000FFCF8091F6020895089522E020934F
:104B4000E9002FEF3091E800215035FD06C035ED2A
:104B50003A95F1F700002111F5CF2091E80025FFEB
:104B60000BC040E050E066E070E00E948428809135
:104B7000E8008E778093E8000895CF93DF9321E0DB
:104B80002093E9002FEF3091E800215035FD06C059
:104B900035ED3A95F1F700002111F5CF2091E800AD
:104BA00025FF14C0EC0140E050E068E070E00E9496
:104BB00084288091E8008E778093E80088E0FE01E9
:104BC000AEEEB2E001900D928A95E1F7DF91CF91C0
:104BD00008958093EA027093EC026093EB02809157
:104BE0003203843001F582E08093E9008FEF9091E9
:104BF000E800815095FD06C095ED9A95F1F700000B
:104C00008111F5CF8091E80085FF0DC040E050E0B4
:104C100063E070E08AEE92E00E9484288091E800D0
:104C20008E778093E8000895BC0184E00C94E92518
:104C3000BC0183E00C94E92589EC9DE00E94EB0720
:104C400080913103811109C00E94112A0E94732AA8
:104C50008091E20084608093E200089585EC9DE0FD
:104C60000E94EB0710923103089581EC9DE00E94B1
:104C7000EB070C94A3248DEB9DE00E94EB07609161
:104C80002E0381E0611101C080E00C948E2489EB39
:104C90009DE00E94EB079091320381E0943009F08F
:104CA00080E060912E030C9493242091E9022F5F01
:104CB000822F62E30E94282D992319F02093E902A4
:104CC00008951092E9028091ED02882371F180919C
:104CD0003203843041F58091E9008F702091EC001F
:104CE000922F917020FD90E8892B93E09093E9003A
:104CF0009091EB0090FF14C09091EE0097FF10C0D0
:104D00009091E80095FF03C01092F100F9CF9091C7
:104D1000E80090FF05C09091E8009E779093E8002E
:104D20008F708093E9001092ED02089542E061ECEB
:104D300081E00E948A2942E261EC82E00E948A2995
:104D400042E261EC83E00E948A299091320381E083
:104D5000943009F080E060912E030C949C248091A3
:104D60003403833009F45FC030F4813071F0823055
:104D700009F498C008958A3009F484C08B3009F48E
:104D80006AC0893009F0A6C020C080913303813AFF
:104D900009F0A0C08091E800877F8093E8008091AF
:104DA000370390913803892B21F468E08EEE92E06E
:104DB00003C060E080E090E070E00E94CF28809126
:104DC000E8008B778093E800089580913303813267
:104DD00009F080C08091370390913803029708F062
:104DE00079C08091E800877F8093E8008091E80097
:104DF00082FD05C0809132038111F8CF6BC0809194
:104E0000F2009091F300029731F48091F10081302B
:104E100011F0863021F48091F1008093F6028091A8
:104E2000E8008B7753C080913303813A09F052C078
:104E30008091370390913803892B09F04BC0809102
:104E4000E800877F8093E8008091E80080FFFCCF36
:104E50008091180136C0809133038132D9F5809159
:104E6000370390913803892BA9F58091E800877F5B
:104E70008093E8000E94BF29809135038093180138
:104E80000C941D0F80913303813221F58091E8004D
:104E9000877F8093E8000E94BF298091360380932A
:104EA000F702089580913303813AA1F48091E800DC
:104EB000877F8093E8008091E80080FFFCCF80919D
:104EC000F7028093F1008091E8008E778093E800EC
:104ED0000C94BF2908959FB7F8941092ED029FBFDC
:104EE00090913203943009F057C09091E9009F707F
:104EF0003091EC00232F217030FD20E8922B23E02D
:104F00002093E9002091EB0020FF43C02091EE00A8
:104F100027FF3FC02091E802222321F02091E800E2
:104F200025FF37C01092E80226E03091E80035FDF9
:104F300015C030913203343061F53091EB0035FD0E
:104F400028C0215021F481E08093E80222C0EFE9DB
:104F5000FFE03197F1F700C00000E7CF8093F10048
:104F60008091E80085FD0AC08091E80080FFFCCFB9
:104F70008091E8008E778093E80006C08FB7F894A0
:104F800021E02093ED028FBF9F709093E90080E0B5
:104F900008959F709093E9008FEF089584B7877FFD
:104FA00084BF0FB6F894A8958091600088618093C3
:104FB0006000109260000FBE90E080E80FB6F89499
:104FC00080936100909361000FBE0C949E240E9418
:104FD000112A0E94732AE2EEF0E0808184608083CF
:104FE00078940C940D2D8CE091E00C94AA23809180
:104FF00032038530C9F485EB9DE00E94EB07809178
:105000003203853079F40E94F124809130038823A3
:10501000B1F30E94B024882391F30E946E280E946D
:105020001D0FEDCF0C941C25089508950C9418289D
:10503000292F332723303105C9F060F421303105A1
:1050400081F02230310509F041C08BE590E02BEF73
:105050003DE040C021323105E1F02232310531F12D
:1050600035C082E190E026E53EE034C099278130EA
:10507000910549F028F0029749F5EDECFDE005C0F7
:10508000E7EFFDE002C0E5EEFDE0849190E09F01D6
:1050900021C063307105D0F4660F771FFB01E55026
:1050A000FE4F2081318189E090E014C063307105AA
:1050B00068F4FB01EE0FFF1FEB50FE4F20813181A2
:1050C000FB01EE50FE4F808190E004C080E090E054
:1050D00020E030E0FA0131832083089584E189BD26
:1050E00086E189BD09B400FEFDCF8091D8008F7D97
:1050F0008093D8008091E00082608093E0008091EE
:10510000E00081FDFCCF0895CF92DF92EF92FF92F5
:105110000F931F93CF93DF93EC018B017A010E94D1
:10512000DE29811133C0E114F10439F0F7018081E7
:105130009181081B190BC80FD91FC12CD12C011547
:10514000110519F18091E80085FD16C08091E800F5
:105150008E778093E800E114F10449F0F701808133
:105160009181C80ED91ED182C08285E00FC00E94F5
:10517000DE29882321F30AC089918093F100015030
:105180001109FFEFCF1ADF0ADACF80E0DF91CF916C
:105190001F910F91FF90EF90DF90CF900895209195
:1051A000390330913A032617370748F06115710526
:1051B00039F42091E8002E772093E80001C0B9016E
:1051C000FC0120E06115710569F1809132038823AB
:1051D000E1F18530E1F18091E80083FD3AC08091F2
:1051E000E80082FD2CC08091E80080FFEBCF809129
:1051F000F2009091F3006115710551F0883091052E
:1052000038F421912093F100615071090196F3CF98
:1052100021E0089709F020E08091E8008E778093E4
:10522000E800D0CF2111D1CF0AC08091320388236A
:1052300061F0853061F08091E80083FD0AC08091C3
:10524000E80082FFF2CF80E0089582E0089583E0D5
:10525000089581E008952091390330913A0326178B
:10526000370748F06115710539F42091E8002E7771
:105270002093E80001C0B901FC0120E0611571052F
:1052800081F180913203882309F43EC0853009F40E
:105290003DC08091E80083FD3BC08091E80082FD25
:1052A0002DC08091E80080FFE9CF8091F2009091BD
:1052B000F3006115710559F08830910540F424918F
:1052C0002093F1003196615071090196F2CF21E0EF
:1052D000089709F020E08091E8008E778093E8003D
:1052E000CDCF2111CECF0AC080913203882361F047
:1052F000853061F08091E80083FD0AC08091E8006C
:1053000082FFF2CF80E0089582E0089583E008955F
:1053100081E00895982F973068F59093E9009817E9
:1053200039F07091EC002091ED005091F00003C035
:10533000242F762F50E021FD02C09F5FECCF3091EB
:10534000EB003E7F3093EB003091ED003D7F3093DA
:10535000ED003091EB0031603093EB007093EC0086
:105360002093ED005093F0002091EE0027FDE5CF53
:1053700080E008958F708093E90081E00895809126
:10538000330387FF11C08091E80082FD05C0809142
:1053900032038111F8CF11C08091E8008B770BC0E8
:1053A00080913203882349F08091E80080FFF8CF94
:1053B0008091E8008E778093E80008952091E400C2
:1053C0003091E50095E64091EC00842F817040FF1C
:1053D00023C08091E80080FD1DC0809132038823A6
:1053E00099F0853099F08091EB0085FD11C04091D6
:1053F000E4005091E5002417350729F3915011F08E
:105400009A01E1CF84E0089582E0089583E0089551
:1054100081E0089580E008954091E80042FFDDCFEB
:1054200008950E94822A0E948A2AE0EEF0E080819C
:1054300081608083E8EDF0E080818F77808319BC04
:10544000A7EDB0E08C918E7F8C9380818F7E8083DE
:105450001092310308950F931F93CF93DF930E940F
:10546000822A0E948A2AC8EDD0E088818F778883BB
:1054700088818068888388818F7D8883E7EDF0E06C
:1054800080818068808319BC1092320310922E03B1
:105490001092300310922F0300EE10E0F80180818B
:1054A0008B7F808388818160888342E060E080E038
:1054B0000E948A29E1EEF0E080818E7F8083E2EE17
:1054C000F0E0808181608083808188608083F80142
:1054D00080818E7F8083888180618883DF91CF91F6
:1054E0001F910F910895E8EDF0E080818F7E808319
:1054F000E7EDF0E080818160808381E0809331037B
:105500000C942B2AE8EDF0E080818C7F8083109250
:10551000E20008951092DA001092E10008951F92BF
:105520000F920FB60F9211240BB60F922F933F9349
:105530004F935F936F937F938F939F93AF93BF939B
:10554000EF93FF938091E10082FF0BC08091E20016
:1055500082FF07C08091E1008B7F8093E1000E9471
:1055600055268091DA0080FF1FC08091D80080FF0F
:105570001BC08091DA008E7F8093DA008091D90081
:1055800080FF0DC084E189BD86E189BD09B400FEBC
:10559000FDCF81E0809332030E941C2605C019BC18
:1055A000109232030E942E268091E10080FF19C0E4
:1055B0008091E20080FF15C08091E2008E7F809391
:1055C000E2008091E20080618093E2008091D80047
:1055D00080628093D80019BC85E0809332030E94DA
:1055E0003B268091E10084FF30C08091E20084FF7F
:1055F0002CC084E189BD86E189BD09B400FEFDCFE0
:105600008091D8008F7D8093D8008091E1008F7EBB
:105610008093E1008091E2008F7E8093E200809190
:10562000E20081608093E20080912E03882311F0D4
:1056300084E007C08091E30087FD02C081E001C0E3
:1056400083E0809332030E9447268091E10083FF2C
:1056500029C08091E20083FF25C08091E100877F0F
:105660008093E10082E08093320310922E038091B8
:10567000E1008E7F8093E1008091E2008E7F809335
:10568000E2008091E20080618093E20042E060E00D
:1056900080E00E948A298091F00088608093F00069
:1056A0000E943526FF91EF91BF91AF919F918F910D
:1056B0007F916F915F914F913F912F910F900BBE12
:1056C0000F900FBE0F901F9018951F920F920FB65C
:1056D0000F9211240BB60F922F933F934F935F932A
:1056E0006F937F938F939F93AF93BF93CF93DF93EA
:1056F000EF93FF93C091E900CF708091EC00D82F19
:10570000D17080FDD0E81092E9008091F000877F91
:105710008093F00078940E94AD2B1092E900809164
:10572000F00088608093F000CD2BCF70C093E9002B
:10573000FF91EF91DF91CF91BF91AF919F918F91A9
:105740007F916F915F914F913F912F910F900BBE81
:105750000F900FBE0F901F9018951F93CF93DF935C
:10576000CDB7DEB7AA970FB6F894DEBF0FBECDBF98
:10577000E3E3F3E08091F100819323E0EB33F20760
:10578000C9F70E94AF268091E80083FF2EC1809167
:10579000330390913403492F50E04A30510508F00B
:1057A00024C1FA01E85AFF4F0C94482D803821F0AB
:1057B000823809F01AC108C080912F0390913003FC
:1057C000992389F082600FC0809137038F708730F2
:1057D00008F00BC18093E9008091EB0085FB8827DE
:1057E00080F91092E9009091E800977F9093E8008B
:1057F0008093F1001092F100D1C0282F2D7F09F085
:10580000F4C0882319F0823061F0EFC08091350335
:10581000813009F0EAC0933009F080E080933003D2
:105820002EC08091350381112AC0809137038F707B
:105830002FEF280F263008F0D8C08093E900209180
:10584000EB0020FF1CC0933021F48091EB008062BC
:1058500014C09091EB0090619093EB0021E030E058
:10586000A90102C0440F551F8A95E2F74093EA0050
:105870001092EA008091EB0088608093EB00109218
:10588000E9008091E800877F8093E8000E94BF29AB
:10589000ACC08111AAC0109135031F778091E3003D
:1058A0008078812B8093E3008091E800877F80934C
:1058B000E8000E94BF298091E80080FFFCCF809122
:1058C000E30080688093E300111102C082E001C010
:1058D00083E08093320389C08058823008F085C00D
:1058E00080913503909136038C3D53E0950779F50F
:1058F00083E08A838AE289834FB7F894DE011396A6
:1059000020E03EE051E2E32FF0E050935700E491B5
:1059100020FF03C0E295EF703F5FEF708E2F90E0A5
:10592000EA3010F0C79601C0C0968D939D932F5F0B
:10593000243149F74FBF8091E800877F8093E800CA
:105940006AE270E0CE0101960E94CF2816C06091F5
:10595000370370913803AE014F5F5F4F0E941628E6
:10596000BC01892B09F441C09091E800977F909386
:10597000E80089819A810E942B298091E8008B7729
:105980008093E80032C0803881F58091E800877FFD
:105990008093E80080912E038093F1008091E800CD
:1059A0008E7772CF811121C080913503909136039B
:1059B00099270297D4F48091E800877F8093E800CC
:1059C0008091350380932E030E94BF2980912E037E
:1059D000811106C08091E30087FD02C081E001C013
:1059E00084E0809332030E9496268091E80083FF32
:1059F0000AC08091E800877F8093E8008091EB00E7
:105A000080628093EB00AA960FB6F894DEBF0FBEBB
:105A1000CDBFDF91CF911F910895CF938091320335
:105A20008823A1F0C091E900CF709091EC00892FFC
:105A3000817090FD80E8C82B1092E9008091E80009
:105A400083FD0E94AD2BCF70C093E900CF910895E4
:105A5000991B79E004C0991F961708F0961B881FC0
:105A60007A95C9F78095089597FB072E16F4009450
:105A700007D077FD09D00E94512D07FC05D03EF4D8
:105A8000909581959F4F0895709561957F4F0895EA
:105A9000EE0FFF1F0024001C0BBE0790F691E02DB7
:105AA0000994AA1BBB1B51E107C0AA1FBB1FA61765
:105AB000B70710F0A61BB70B881F991F5A95A9F7B7
:105AC00080959095BC01CD010895FB01DC0104C0D7
:105AD0008D910190801921F441505040C8F7881BE6
:105AE000990B0895F999FECF92BD81BDF89A992737
:105AF00080B50895A8E1B0E042E050E00C94A62DF6
:105B0000262FF999FECF92BD81BDF89A019700B476
:105B1000021639F01FBA20BD0FB6F894FA9AF99A16
:105B20000FBE08950396272F0E94812D0E94802D7D
:105B3000252F0E94812D242F0C94812D0196272F33
:105B40000E94812D0C94802DDC01CB01FC01F99980
:105B5000FECF06C0F2BDE1BDF89A319600B40D92B9
:0C5B600041505040B8F70895F894FFCF72
:105B6C00C8009B02280850011E0A14019A25BD2565
:105B7C009E25182614269D2501E200E900EA00B5B1
:105B8C0000B600B700CD008301CC008A01920194CD
:105B9C00012102230224022502260227022A02B333
:105BAC0000B4006F007000818283E200E900EA001B
:105BBC00B500B600B700CD008301CC008A0192017C
:105BCC0094012102230224022502260227022A0222
:105BDC00B300B4006F007000818283F76766656460
:105BEC0063626160C1C0979695949392919037F1DE
:105BFC00F2F3F4F5F63F3F3F006D6B5F64656C614B
:105C0C0079006D6B5F696E74657276616C006D6B9B
:105C1C005F6D61785F7370656564006D6B5F74694F
:105C2C006D655F746F5F6D6178006D6B5F77686534
:105C3C00656C5F6D61785F7370656564006D6B5F3B
:105C4C00776865656C5F74696D655F746F5F6D61B6
:105C5C007800407B22050F8A0E680E0D0E260E3F33
:025C6C000E0028
:00000001FF
